:020000040000FA
:0400000006303A2864
:08000800A000030EA100831209
:100010008B1C32288B1031181428B11C3228643004
:10002000010203183128182800001628172818285C
:1000300019281A281B281C281D281E281F283110A3
:10004000B114A810031005190314AA0DA90DA80DC9
:10005000B00B322831152A08AF002908AE00280855
:10006000AD00B11081010B11210E8300A00E200EF6
:02007000090085
:0C007400203084008001840A6030040207
:10008000031C3C281230B00095218316FF239000FA
:10009000831283160C308505870183128501870141
:1000A000073099000030831691009F008312C830FA
:1000B00083168100831231309000003083168C004B
:1000C000831210308B00ED2181018E018F010B1105
:1000D0008B100B108C018B177B2031199120B30BE7
:1000E0007928031085190314B90DF030390203196A
:1000F0000A2101226C286400311808000B1D080039
:100100000B11B11031141230B000051D8C283214BF
:10011000831601138312080032108316011783120D
:10012000080031110130B7008B13203037078316D8
:100130009B001C141A088312A400A500C030A50659
:100140001030370783169B001C141A088312A30073
:100150000030370783169B001C141A088312A20074
:100160008B17321CB92822090339A200A309A4095C
:10017000A50922082D02031D042923082E02031DB0
:10018000042924082F02031D042901303702031D0E
:10019000CE283D18CE283D143E14A321023037024C
:1001A000031DD728BD18D728BD143E14AA2103303B
:1001B0003702031DE0283D19E0283D153E14B1210A
:1001C00004303702031DE928BD19E928BD153E1486
:1001D000B82105303702031DF2283D1AF2283D16DA
:1001E0003E14BF2106303702031DFB28BD1AFB2831
:1001F000BD163E14C62107303702031D04293D1BDE
:1002000004293D173E14CD21B70A083037020318E0
:10021000080094280130B600B300B400B500B70060
:1002200085018701B1137B20B30B48290310851981
:100230000314B90DF030390203196F29B40B4829A2
:10024000013037020319D521023037020319D821B2
:10025000033037020319DB21043037020319DE2192
:10026000053037020319E121063037020319E42172
:10027000073037020319E7219630B4000330370204
:1002800032300319B4000430370232300319B4009D
:10029000311D13293111321C52292D090339AD00AA
:1002A000AE09AF092F1CB1132F1C1329B11B132941
:1002B0002E181329B1178B1320303707BB002F08D6
:1002C000BA00822110303707BB002E08BA00822105
:1002D00000303707BB002D08BA0082218B1785013B
:1002E0008701B70AB60108303702031C1329ED2134
:1002F00008003E1C08003E101030BB003D08BA004C
:10030000822108008B133A0883161C159A003B08BB
:100310009B0055309D00AA309D009C1464009C18E1
:100320008E291C1183128B170800831610309B0036
:100330001C141A088312BD00FF30D000D415D51547
:10034000D615D7150800BD103D11BD110230CE00E5
:10035000D20008003D103D11BD110130CE00D20089
:1003600008003D10BD10BD118230CE00D200080043
:100370003D10BD103D114130CE00D2000800BD122D
:100380003D13BD130030CF00D30008003D123D13D4
:10039000BD130230CF00D30008003D12BD12BD13C3
:1003A0000130CF00D30008000800013085060800A6
:1003B00002308506080001308506080002308506F7
:1003C000080030308506080010308506080020300F
:1003D000850608002230850608003D18A321BD18B7
:1003E000AA213D19B121BD19B8213D1ABF21BD1A5D
:1003F000C6213D1BCD21BD1BD4213D080319A321DE
:1004000008008F08031908008F0196308E00D00F66
:10041000BB2AD00ABD1A332A521C332A521F242A5F
:10042000D41C152AD4015415412A541D1A2AD4016A
:10043000D415412AD41D1F2AD4015416412A541E12
:10044000412AD401D414412A541D292AD401541616
:10045000412AD41D2E2AD4015416412A541E412A61
:10046000D401D414412AD41C382AD4015415412A69
:10047000541D3D2AD401D415412A541E412AD401C9
:100480005415BD1A6A2AD21C6A2AD21F5B2AD51CAF
:100490004C2AD5015515782A551D512AD501D51557
:1004A000782AD51D562AD5015516782A551E782A40
:1004B000D501D514782A551D602AD5015516782AFC
:1004C000D51D652AD5015516782A551E782AD501DD
:1004D000D514782AD51C6F2AD5015515782A551DB3
:1004E000742AD501D515782A551E782AD5015515B7
:1004F000531C892A561D7F2AD6015616972AD61DC7
:10050000842AD6015616972A561E972AD601D61443
:10051000972AD61C8E2AD6015615972A561D932A3D
:10052000D601D615972A561E972AD6015615D31CE2
:10053000A82A571D9E2AD7015716B62AD71DA32AC7
:10054000D7015716B62A571EB62AD701D714B62A8E
:10055000D71CAD2AD7015715B62A571DB22AD70185
:10056000D715B62A571EB62AD701571579214E0836
:10057000D2004F08D3005008D1000C305405031DA1
:1005800085100C305505031D05100C305605031D54
:1005900085120C305705031D051251080E02031871
:1005A000E52A12305405031D851412305505031D2C
:1005B000051412305605031D851612305705031D0C
:1005C0000516FF305002031908008F08031D0800AC
:1005D0007B2051080E02031CE52A18305405031D28
:1005E000851006305405031D851418305505031D6C
:1005F000051006305505031D051418305605031D5A
:10060000851206305605031D851618305705031D43
:0C061000051206305705031D05160800F2
:084000000E00030006000000A1
:02400E00CC01E3
:10420000010003000300030003000200020002009B
:1042100002000000000000000000FF00FF00FF009F
:10422000000000000000000000000000000000008E
:104230000000C000C000C000C000FF00FF00FF0081
:104240000100C300F300CF00FF00C300F300CF0064
:10425000FF00C300F300CF00FF00FF00FF00FF00DE
:10426000FF00FF00FF00FF00FF00FF00FF00FF0056
:10427000FF00FF00FF00FF00FF00FF00FF00FF0046
:10428000FF00FF00FF00FF00FF00FF00FF00FF0036
:10429000FF00FF00FF00FF00FF00FF00FF00FF0026
:1042A000FF00FF00FF00FF00FF00FF00FF00FF0016
:1042B000FF00FF00FF00FF00FF00FF00FF00FF0006
:1042C000FF00FF00FF00FF00FF00FF00FF00FF00F6
:1042D000FF00FF00FF00FF00FF00FF00FF00FF00E6
:1042E000FF00FF00FF00FF00FF00FF00FF00FF00D6
:1042F000FF00FF00FF00FF00FF00FF00FF00AA001B
:00000001FF
